:100000008A150028FF3FFF3F03138312F8010830D1
:10001000FC00700DF80D7408F80203181128F80799
:100020000310F00DFC0B0928080000000000080078
:10003000040803138316C700831220088400841366
:1000400000088316C600C6134613460880004708FA
:1000500084000800031383127008F100F0010830D7
:10006000FC007108F40C03183928FC0B3228F1014C
:10007000003403103E28F40C0318F107F10CF00CC7
:10008000FC0B3B28080003138316C4014308093CFA
:1000900003186A280A30F4004308F00004207008AE
:1000A0008316C4007008C500C50D4510C50D451068
:1000B000C50D4510C50D45104508C4000A30F400B3
:1000C0004308F00004207808F00070088316450407
:1000D000C4006C284308C4004408F000080003135F
:1000E00083164308C5004508F100C50A440884008A
:1000F000C40A0008F00071088400700880007108CC
:1001000084000008F0007008031D73284308F00005
:100110000800031383164308C40044088400C40A7B
:100120000008F0007008031D8D2843084402F00009
:100130000130F002F101031CF10308000030031349
:10014000831698180130F1007108003A031DAA289F
:1001500000009E28430883129900080003138312AD
:1001600020088400831380171520001715201820FD
:10017000801315201820001308000830031383167D
:10018000C400C50183122008840083138316440829
:100190000319E42815201520182000131520430802
:1001A0000319D2281820C30D031CD92884178017DF
:1001B000DB28841780130000152000178413001F0C
:1001C000DF288417C403C628C501152018200000A5
:1001D0000013152080171520152045080319F02855
:1001E00000178413001FF228C50115208413801BFB
:1001F0004514152015201520152015201520152033
:10020000152018208417001380134508F0000800FB
:1002100003138312200884008313182080131520F1
:1002200000178413001F122984171520152015208C
:10023000152080171520080003138312F801F90117
:100240001030FC00710DF80DF90D7408F8027508F6
:10025000031C750FF902031834297408F807750890
:100260000318750FF9070310F00DF10DFC0B22298F
:1002700008000313831222088A0023088200080062
:10028000083003138316C000C101831220088400C4
:10029000831383164008003C0318642915200000CE
:1002A0008017152041080319552900178413001FD2
:1002B0005729801B0314801F0310C10D152018201F
:1002C00084170013C0034929801715203F0803191C
:1002D0006A2918203F0803196E2980130000152091
:1002E00000178413001F722984171520182000138B
:1002F0001520182080134108F00008000F30031368
:1003000083163F05C0003F08F000F00CF013F00C1E
:10031000F013F00CF013F00CF0130A30F4002A2064
:1003200083164008F0070800031383163F08C30034
:10033000432070088312A400F0307005A500A601C8
:100340000030A6050030A6000430F2002508F000B9
:100350002608F10072080319B429F10CF00CF1130E
:10036000711BF117FF3FAB297008A5007108A600AB
:100370003030F0070318F10A7008A5007108A600D4
:1003800027088400700880000F302405A500A6010E
:100390000030A6050030A60030302507F200260800
:1003A0000318013FF3000030F3077208A50073083B
:1003B000A600270AF000700884007208800002304E
:1003C0002707F00070088400280880000330270702
:1003D000F0007008840080010800031383163F08B2
:1003E000C100410884000008F00070080319FA29D0
:1003F000C10AF1294108F100C10A40088400C00A7D
:100400000008F00071088400700880007108840002
:100410000008F0007008031DFA293F08F0000800EA
:100420000313831229088316C3003F08C4006F20FA
:1004300070088312A90070088316C3008920700811
:10044000C100C001400883122907840000088316F8
:10045000C3009E208316C00A80304006F000803022
:1004600041067002031C222A0800AE20A430C300FB
:10047000BD204008F000F1017008C300BD2000302D
:10048000F4000130F5003F08F0004008F1001C21A5
:100490007808F0007908F10070088316C300BD20C9
:1004A0000330FB00FF30FA00FB0B572A5A2AFA0BE5
:1004B000572A542A9630FA00FA0B5C2A00004108A9
:1004C000C300BD200821C20180304206F000803008
:1004D000033A70020318852A0330FB00FF30FA004C
:1004E000FB0B732A762AFA0B732A702A9630FA00CD
:1004F000FA0B782A0000C301BD2070080319822A74
:10050000AE20832A852AC20A642A08000E3003130B
:100510008312FA00FA0B8A2A0000080003138312E0
:100520002230FC00F801F901FA01FB01FC03031978
:10053000C42A0310FB0CFA0CF90CF80CF30CF20CA7
:10054000F10CF00C031C962AFC030319B62A74085C
:10055000F80775080318750FF90776080318760F62
:10056000FA0777080318770FFB079A2A7408F80729
:1005700075080318750FF90776080318760FFA0740
:1005800077080318770FFB0708000313831286010F
:100590008316860185309F00FF3083128500FF306F
:1005A00083168500831287018316870108000313D1
:1005B0008316031383163908F200B90A3A08F000CB
:1005C0003B08F100BA0A0319BB0A70088312A300A2
:1005D0007108A2000A08A1003921F00021088A0050
:1005E0007208840070088000720884000008F0001F
:1005F00070080319FC2AD72A08004D3469346B347B
:1006000072346F3443342034383437343634203441
:1006100032343434363434345F3432342E34433468
:100620000A340D34203400340800031383122908DF
:100630008400800108218230FB00FF30FA00FB0BB0
:10064000222B252BFA0B222B1F2B8730FA00FA0BBB
:10065000272B00000000AE20D030C300BD20C30116
:10066000BD20AE20D130C300BD200130BF004021ED
:1006700070088312A500A60125088316BF007E21FD
:1006800070088312B00001308316BF00402170084B
:100690008312A500A60125088316BF007E217008DD
:1006A0008312AF0001308316BF004021700883120F
:1006B000A500A60125088316BF007E2170088312BD
:1006C000AE0001308316BF00402170088312A500E0
:1006D000A60101308316BF00402170088312A500D7
:1006E000A60125088316BF007E2170088312AC0086
:1006F00001308316BF00402170088312A500A601B7
:1007000025088316BF007E2170088312AB00831674
:10071000BF01402170088312A500A6012508831699
:10072000BF007E2170088312AA002908840080017E
:100730002F30A8002A088316BF00942129088316A9
:10074000BF00831227088316C000ED212F308312CB
:10075000A8002B088316BF00942129088316BF0028
:10076000831227088316C000ED2120308312A800D1
:100770002C088316BF00942129088316BF0083121A
:1007800027088316C000ED21831229088316BF00B5
:1007900010220930C3009E202908840080014830BF
:1007A000A8002E088316BF00942129088316BF00D5
:1007B000831227088316C000ED214D308312A80054
:1007C0002F088316BF00942129088316BF008312C7
:1007D00027088316C000ED2153308312A80030088B
:1007E0008316BF00942129088316BF0083122708AF
:1007F0008316C000ED21831229088316BF00102242
:100800000930C3009E200800031383163B088400B0
:10081000203080002030840A8000840A8000840A0E
:100820008000840A80000130BC003A08003C031DAF
:100830001B2C3908093C03181E2CBC0A3A08003C42
:10084000031D242C3908633C0318272CBC0A3A08E2
:10085000033C031D2D2C3908E73C0318302CBC0A3F
:100860003A08273C031D362C39080F3C0318392C55
:10087000BC0A05303B07F000700884008001840347
:100880003C08003C0318692C0A30F400F5013908D3
:10089000F0003A08F1001C217808F0007908F10016
:1008A00070088000000883163902F0000030031C35
:1008B000013F3A02F1000A30F400F5011C217008F2
:1008C0008316B9007108BA00303080078403BC0376
:1008D000402C0800031383163908C30089207008D0
:1008E000BC007108BD00BA01BB0180303B06F000BE
:1008F00080303D067002031D7F2C3C083A0203182D
:10090000982C831231088316BF0083123208831695
:10091000C0003A08390784000008C100352283125C
:10092000B10A0319B20A8316BA0A0319BB0A752C55
:100930000800031383129F01C0309F0483161F1702
:100940009F173908F000F00D7010F00D7010F00DC9
:100950007010700883129F041F1486221F151F1D1C
:10096000B32C0000AF2C1F100830F2001E08F0005E
:10097000F10172080319C12CF00DF10D7010FF3F49
:10098000BA2C83161E08F0040030F1040800003071
:10099000031383128C1A0130F1007108F000080073
:1009A000031383121A088316B9008312981CDA2CD9
:1009B0001812181683163908F00008000A340D348E
:1009C000463469346E3420346434653420347034F1
:1009D00072346F3467340A340D34003408000A343A
:1009E0004C34653463347434753472346534203473
:1009F00045344534503452344F344D3420346E3401
:100A00000D3400340800AE20A430C300BD203A08E5
:100A1000F000F1017008C300BD200030F400013087
:100A2000F5003908F0003A08F1001C217808F000C0
:100A30007908F10070088316C300BD20AE20A530F0
:100A4000C300BD20BF0140217008BB0008213B0846
:100A5000F0000800D03003138316BB000730BC0041
:100A6000BD01BE010530F4003B08F0003C08F10078
:100A70003D08F2003E08F30074080319462DF30CFC
:100A8000F20CF10CF00CF313FF3F3D2D7008BB008E
:100A90007108BC007208BD007308BE003908F4007C
:100AA0003A08F500F601F7018E2270088316BB00A4
:100AB0007108BC007208BD007308BE003B083C040E
:100AC0003D043E040319702D0130BB02031CBC021F
:100AD000031CBD02031CBE020000000000005E2DCE
:100AE00008004D3003138312B3006930B4006B303B
:100AF000B5007230B6006F30B7004330B800203018
:100B0000B9003830BA003730BB003630BC00203076
:100B1000BD005030BE005730BF004D30C000203007
:100B2000C1007430C2006530C3007330C40074303B
:100B3000C5002030C6003030C7003430C800203037
:100B4000C9000A30CA000D30CB00CC013330A900F7
:100B50002E30CD002E30CE002E30CF002E30D000E3
:100B60002E30D1002E30D2002E30D3002E30D400C3
:100B70002E30D5002E30D6002E30D7002E30D800A3
:100B80002E30D9002E30DA002E30DB002E30DC0083
:100B90002E30DD002E30DE002E30DF002E30E00063
:100BA0002E30E1002E30E2002E30E3002E30E40043
:100BB0002E30E5002E30E6002E30E7002E30E80023
:100BC000E9014D30A7002F308316A0002F30A1007F
:100BD0002F30A2004430A3004830A4004D30A500BF
:100BE0005330A600A701080003138316981690300F
:100BF0008312980083168717071383128C1E042E06
:100C00001A088316BD00FD2D031383160800031375
:100C10008316390884000008BA00BA133A133A0858
:100C20008000841704088312A00080170017841323
:100C3000001F182E0800FF3FFF3FFF3FFF3FFF3F11
:100C4000FF3FFF3FFF3FFF3FFF3FFF3FFF3FFF3FB4
:100C5000FF3FFF3FFF3FFF3FFF3FFF3FFF3FFF3FA4
:100C6000FF3FFF3FFF3FFF3FFF3FFF3FFF3FFF3F94
:100C7000FF3FFF3FFF3FFF3FFF3FFF3FFF3FFF3F84
:101000008A1171258A152030A9004D30AA0065305B
:10101000AB007330AC003130AD003D30AE0020305D
:10102000AF00B0012030B1004D30B2006530B300E8
:101030007330B4003230B5003D30B6002030B70018
:10104000B8018A11C5228A15E8308312EA000330FC
:10105000EB0033308316990018158A11F4258A1590
:10106000831229088316B900FD30BA000230BB0094
:101070008A11D7228A1529088316BF008A111022E7
:101080008A150630B9008A1107268A150230FC003D
:10109000FF30FB00FF30FA00FC0B4F285628FB0BFB
:1010A00052285528FA0B52284F284C280630FB00AE
:1010B000FF30FA00FB0B5D286028FA0B5D285A28E8
:1010C0000A30FA00FA0B622800008A1115238A15EB
:1010D000B101B201EC01ED010313831220303202A1
:1010E000031D7428003031020318F0293208F00083
:1010F000F1017008A5007108A60070088316B900F8
:101100007108BA00831229088316BB008A110424CF
:101110008A15831229088316BF008A1110228A15A6
:10112000FF3083123105F0003208F1000030F10584
:101130007008A5007108A60070088316B900710830
:10114000BA00831229088316BB008A1104248A1569
:10115000831229088316BF008A1110228A150930CC
:10116000C3008A119E208A158A1115238A15290821
:101170008316B9008A116A248A15831231088316EE
:10118000BF00831232088316C0000930C1008A11E3
:1011900035228A158312B10A0319B20A8316B901DE
:1011A0008A1199248A1570088312A5007108A60077
:1011B000A9308316BF008A1110228A1583122508D0
:1011C0008316B900831226088316BA0083122908F1
:1011D0008316BB008A1104248A15831229088316FA
:1011E000BF008A1110228A150930C3008A119E207F
:1011F0008A1529088316B9008A116A248A15831270
:1012000031088316BF00831232088316C0000930EC
:10121000C1008A1135228A158312B10A0319B20A54
:1012200001308316B9008A1199248A157008831237
:10123000EE007108EF00B1308316BF008A11102252
:101240008A1583126E088316B90083126F088316FD
:10125000BA00831229088316BB008A1104248A1558
:10126000831229088316BF008A1110228A150930BB
:10127000C3008A119E208A1529088316B9008A1195
:101280006A248A15831231088316BF00831232083C
:101290008316C0000D30C1008A1135228A158312D1
:1012A000B10A0319B20A0D308316C3008A119E20B9
:1012B0008A158A11C7248A157008031964298A11AE
:1012C000D0248A157008A80003138316CD29643032
:1012D0008312EA000030EB00E32903138312E830A5
:1012E000EA000330EB00E32903138312A030EA0085
:1012F0000F30EB00E3290313831229088316B9008A
:10130000DE30BA000430BB008A11D7228A152908C2
:101310008316BF008A1110228A158D29013083128D
:101320003102EC000030031C013F3202ED00B1013C
:10133000B20129088316B900EF30BA000430BB00AF
:101340008A11D7228A1529088316BF008A11102214
:101350008A1583126D083202031DB0296C08310210
:101360000318C92931088316B9008312320883167D
:10137000BA008A1103258A1570088312A400B10AE5
:101380000319B20A70088316C3008A119E208A15B9
:10139000A929E32903138312E32983162808303A85
:1013A000031967292808313A03196D292808323AA8
:1013B000031974292808513A03197B2928084C3A43
:1013C00003198E29CA2983126A088316B900831269
:1013D0006B088316BA008A112A258A15A8016C2881
:1013E00003138316F229FF3FFF3FFF3FFF3FFF3FFD
:02400E00FA3F77
:00000001FF
